S00E0000626C696E6B792E737265638D
S11300000C943E000C945B000C945B000C945B001D
S11300100C945B000C945B000C945B000C945B00F0
S11300200C945B000C945B000C945B000C945B00E0
S11300300C945B000C945B000C945B000C945B00D0
S11300400C945B000C945B000C945B000C945B00C0
S11300500C945B000C945B000C945B000C945B00B0
S11300600C945B000C945B000C945B000C945B00A0
S11300700C945B000C945B000C945B0011241FBE79
S1130080CFEFD0E1DEBFCDBF11E0A0E0B1E0EEE5FF
S1130090F1E002C005900D92A030B107D9F711E04C
S11300A0A0E0B1E001C01D92A030B107E1F70E94C9
S11300B091000C94AD000C940000DF93CF93CDB766
S11300C0DEB728970FB6F894DEBF0FBECDBF6D83A1
S11300D07E838F83988719821A821B821C820BC0AD
S11300E089819A81AB81BC810196A11DB11D89834F
S11300F09A83AB83BC8329813A814B815C818D8156
S11301009E81AF81B885281739074A075B0744F3F6
S113011028960FB6F894DEBF0FBECDBFCF91DF9106
S11301200895DF93CF93CDB7DEB7E4E2F0E08FEF2D
S11301308083E5E2F0E08FEF808368ED79E580E08D
S113014090E00E945D00E5E2F0E0108268ED79E560
S111015080E090E00E945D00ECCFF894FFCFB9
S9030000FC
